:02000000E628F0
:08000800F000030EF200830179
:100010000408F1000B280B1D29280B1185308100E5
:100020004B203808390403191E28B803380FB90AC1
:10003000B90338083904031D1E283516B70B2928C3
:100040003D30B7004308A2004408A3003514351121
:1000500006130C1D44280C11171C34281508A00089
:100060001608A1001710442817141508A200160836
:10007000A3002008A2022108031C210AA3023514B0
:10008000351506173D30B70071088400720E8300E5
:10009000F00E700E090000308A003C0882075228DA
:1000A00064287F28061C61280800BC018613EE30F6
:1000B000BA000230BB00FA30BD000030BE00B510FF
:1000C00008000130BC000800061872288617B51811
:1000D0000800BA033A0FBB0ABB033A083B040319F2
:1000E000B5140800B51C55280230BC00F230C10020
:1000F0000530C200F230C5000530C6000800061CFD
:10010000B028BD033D0FBE0ABE033D083E04031DDB
:100110009028FA30BD000030BE000608803A860004
:10012000351C0800351042082302031D9928410898
:10013000220203189F282208C1002308C200460893
:100140002302031DA52845082202031CAB28220810
:10015000C5002308C6002208C3002308C400080005
:100160004508B3004608B4001530B3020030031C44
:100170000130B4024308B3024408031C440AB40229
:100180004308B1004408B2001530B1020030031C2E
:100190000130B2024108B1024208031C420AB20215
:1001A0003308A8003408A900C830A600A701DA2146
:1001B0002408C7003108A8003208A900C830A600EA
:1001C000A701DA212408C800B51555288301BC0110
:1001D000B5018501860107309F008316023081003A
:1001E0008501860106148615861405168516A63027
:1001F0009800003099000C15830101309000053003
:1002000097008030980086175520B801B901B501D4
:10021000B601051A36140830F5000830F3004130F5
:10022000F40074088400831673089B001C141A08D9
:1002300083128000F30AF40AF50B1129A201A3012D
:100240000B178B160B118B17861306168616B5180F
:100250002729351A3029B51935293518552927295F
:10026000351200308500B5122729B5110830F50088
:100270004130F3000830F4008C1373088400000848
:1002800083169A0074089B001C158B1355309D0033
:10029000AA309D009C148B171C1183128C1F4E29B1
:1002A000F30AF40AF50B3C292729351046082302E6
:1002B000031D5C2945082202031C62294508A2008F
:1002C0004608A30042082302031D682941082202B0
:1002D00003186E294108A2004208A3002208AF00BB
:1002E0002308B0004308AF024408031C440AB002CC
:1002F000031C8129A530AD004708AB000130AC00DC
:100300008E299630AD004808AB000230AC00AF0932
:10031000B0092F0FB003B00AAF0030040030300234
:10032000031D942915302F02031CA7291530AF0295
:100330000030031C0130B0022F08A8003008A900CB
:100340002B08A600A701DA212408AE00AD29C3308E
:10035000AD00C630AE000030AC00FF300C1EAE2940
:1003600099002D080C1EB22999002E080C1EB629E2
:100370009900FF302D062E060C1EBC299900B51AD7
:1003800027292E08963C0318D3292C088500003C09
:1003900003192729061E2729F430B8000130B900B7
:1003A0003512B51627292E08643C031C2729003076
:1003B000850027290630AA000310A80DA90DAA0B55
:1003C000DC29A401A501260827040319FF34013004
:1003D000AA00A71BF029AA0A0310A60DA70DE92958
:1003E0000310A40DA50D2608A8022708031C270A40
:1003F000A9020318022A2608A80727080318270AB3
:10040000A907032A2414AA0303190A2A0310A70C14
:10041000A60CF0290310A80DA90D2608A80227088C
:10042000031C270AA902031C0800240FA503A50A20
:06043000A40025040034C5
:02400E00693F08
:1042000062000400F20005008200070080008000C8
:1042100062000400F20005008200070080008000B8
:00000001FF
